:020000040800F2
:10000000D806002051030008590300085B030008CC
:100010005D0300085F0300086103000800000000A2
:100020000000000000000000000000006303000862
:10003000650300080000000067030008B11A00080B
:100040006B0300086B0300086B0300086B030008D8
:100050006B0300086B0300086B0300086B030008C8
:100060006B0300086B0300086B0300086B030008B8
:100070006B0300086B0300086B0300086B030008A8
:100080006B0300086B0300086B0300086B03000898
:100090006B0300086B0300086B0300086B03000888
:1000A0006B0300086B0300086B0300086B03000878
:1000B0006B0300086B0300086B0300086B03000868
:1000C0006B0300086B0300086B0300086B03000858
:1000D0006B0300086B0300086B0300086B03000848
:1000E0006B0300086B0300086B0300086B03000838
:1000F0006B0300086B0300086B0300086B03000828
:100100006B0300086B0300086B0300086B03000817
:100110006B0300086B0300086B0300086B03000807
:100120006B0300086B0300086B0300086B030008F7
:100130006B0300086B0300086B0300086B030008E7
:100140006B0300086B0300086B0300086B030008D7
:100150006B0300086B0300086B0300086B030008C7
:100160006B0300086B0300086B0300086B030008B7
:100170006B0300086B0300086B0300086B030008A7
:100180006B0300086B0300086B0300086B03000897
:100190006B030008000000006B0300086B030008FD
:1001A0006B0300086B0300086B0300086B03000877
:1001B0006B0300086B0300086B0300086B03000867
:1001C0006B0300086B0300086B0300086B03000857
:1001D0006B0300086B03000800F002F800F0A8F8B9
:1001E00014A696E8000CB244B344DA4501D100F0FD
:1001F0009FF8BAE80F000FA696E83000A5EB0405BB
:1002000004EB0607AAEB0704A7F101074FEA15154F
:100210004FEA3414A4F10104AC4201D300F088F891
:1002200013F0010F18BFFB1A43F0010300F001F8AF
:10023000DBE718471C2E00003C2E0000103A24BFBC
:1002400078C878C1FAD8520724BF30C830C144BF3B
:1002500004680C6070470000704700000023002411
:1002600000250026103A28BF78C1FBD8520728BFC6
:1002700030C148BF0B6070476E2900F0B181702912
:1002800000F0E782662902F08E85652902F08B85F1
:10029000672902F08885612902F0878503681B0AB7
:1002A00028BF41F08001692900F05E81642900F0D7
:1002B0005B81752900F058816F2900F075827829DB
:1002C00000F0B382E92900F00F82E42900F00C82EB
:1002D000F52900F00982EF2900F07282F82900F078
:1002E000B2820368DB0928BF41F08001632900F076
:1002F000CB87732900F0D087E32900F0DB87F3294F
:1003000000F0E087002070471FB502F03FFD01F0CC
:1003100033F804000020002102F022FD401C606040
:100320000020002102F006FDE0601FBD10B510BDE9
:1003300000F0F4FF1146FFF7E7FF01F0A5FF01F021
:10034000D1F803B4FFF7F2FF03BC01F0DDFC0000BD
:100350000948804709480047FEE7FEE7FEE7FEE759
:10036000FEE7FEE7FEE7FEE7FEE7FEE70448054995
:10037000054A064B70470000A51C0008D90100087B
:10038000D8000020D8060020D8020020D802002083
:10039000704753EA020C00F069802DE9F04B4FF0F2
:1003A0000006002B1FBFB3FA83F503FA05F424FA05
:1003B00005F65E4012BF1643B2FA82F502FA05F462
:1003C000C5F120051EBF22FA05FC44EA0C042035C5
:1003D00056EA044C4FEA144418BF641C4FF000085E
:1003E0004FF00009904271EB030C39D3002919BF7B
:1003F000B1FA81F701FA07F6B0FA80F700FA07F6CA
:10040000C7F120071EBF20FA07FC46EA0C0620377A
:10041000B6FBF4FCA7EB0507103F07F01F0BCBF171
:1004200020062CFA06F60CFA0BFB44BFB346002656
:10043000202FA4BF5E464FF0000B5BEA060C08BFFE
:100440004FF0010B19EB0B0948EB0608ABFB027CE4
:1004500006FB02CC0BFB03CCC01B71EB0C01C1E70C
:100460000B46024641464846BDE8F08B13B50843AB
:1004700018BF4FF0FF300146AFF30080BDE81C40CD
:10048000704700000FB4044910B503AA029800F0A9
:10049000BBF810BC5DF814FB70000020704770477B
:1004A0007047704770B5044685690068C10601D57C
:1004B000302600E02026C00707D070BDD4E9012116
:1004C00030469047206A401C20626D1EF6D570BDF4
:1004D00070B5044685690078C00707D170BDD4E9BE
:1004E000012120209047206A401C20626D1EF6D515
:1004F00070BD09684A0501D540B27047C905FCD5F1
:1005000000B2704709684A0501D5C0B27047C905F5
:10051000FCD580B2704770B50C460546012A05D05F
:100520002878800600D5EA69002302E0012305E06F
:100530005B1C934202D2E05C0028F9D1A869E6185E
:10054000C01AA861286A184428622846FFF7AAFF43
:1005500004E0D5E9012114F8010B9047B442F8D327
:100560002846FFF7B5FF70BD2DE9F041064600248F
:1005700010687529314616A510D0FFF7BAFF00287C
:1005800002DA404213A507E031688A0701D512A5B7
:1005900002E0490704D511A5012401E0FFF7B2FFED
:1005A00000210A2206F1240709E0B0FBF2FCB0FBAF
:1005B000F2F302FB1C00303078541846491C002826
:1005C000F3D123462A463046BDE8F04100F055BA43
:1005D000000000002D0000002B00000020000000A3
:1005E00011680268006A530501D508700AE0D30556
:1005F00001D5088006E0130603D5C217C1E9000241
:1006000000E0086001207047074B70B50D467B4441
:1006100000F01DFE0446284600F058FE10B14FF0D1
:10062000FF3070BD204670BD171800002DE9FF5F38
:1006300015468A460446DFF8AC80F8440027D8E91E
:1006400000103E46CDE9001010E03AF816106A4658
:1006500002A800F03FFE411C07D02178890603D58F
:10066000E269391891420DD80744761C207880063B
:1006700002D5E069B84205DDAE42E6DB3AF8160085
:100680000028E2D1A069C01BA0612046FFF70AFF45
:10069000D8E90010CDE90010002017E03AF8181052
:1006A0006A4602A800F016FEB0F1FF3F81460BD06B
:1006B00000250DF1080B05E0D4E901211BF8050028
:1006C00090476D1C4D45F7D308F10100B0428046BC
:1006D000E4DB206A384420622046FFF7F9FEBDE8DB
:1006E000FF9F0000722700002DE9F0418046D21DD7
:1006F00022F007020025D2E90002F52915A614D040
:10070000011E72F1000106DA0023D0EB030063EB57
:10071000020211A608E0D8F800108B0701D50FA639
:1007200002E0490701D50EA601251146002408F173
:10073000240704E000F05CF930323A55641C50EABA
:100740000102F7D12B46324621464046BDE8F04132
:1007500000F093B9000000002D0000002B00000005
:100760002000000030B4002100F1240408E002F071
:100770000705D208303542EA4372DB086554491C4C
:1007800052EA0305F3D10468002310A2250708D517
:1007900004F020040C4304D0C46901230CA2641E9D
:1007A000C46130BC00F069B910B504462146106838
:1007B000FFF7A8FE02462046BDE810400023D1E71F
:1007C000D21D22F00701D1E90023CBE70000000091
:1007D00030000000F0B40D460188090502D5214C17
:1007E0007C4402E01F4C7C440E34002100F12406BE
:1007F00008E002F00F071209E75D42EA03721B09E5
:100800007754491C52EA0307F3D1027800231207F8
:1008100004D5702D06D009B1022311342246F0BC54
:1008200000F02BB901231034F8E770B504460D46EB
:1008300021461068FFF766FE024629462046BDE8BD
:1008400070400023C6E7D21D22F00703D3E900233E
:10085000C0E70368126843F0200303600823C36104
:100860000023B7E7D42500002DE9F05F8946044650
:100870004FF0000ADFF874B1FB44C0F820A0204616
:10088000E1688847002874D0252806D0D4E90121E2
:100890009047206A401C2062F1E700265F46204610
:1008A000E16888472028054607DB312D05D27819F5
:1008B00010F8200C08B10643F1E7B00701D526F087
:1008C0000406C4F81CA00027C4F818A02A2D09D0DB
:1008D000284602F027FA38B304EB8708303DC8F801
:1008E000185019E059F8041B204604EB8702916167
:1008F000E1688847012F054618D1E069002820DA11
:1009000026F020061DE0D8F8180000EB800005EB6B
:1009100040003038C8F818002046E168884705468E
:1009200002F000FA0028EED1012F0AD02E2D08D1B6
:100930002046E16888477F1C0546022F46F02006C6
:10094000C4DBA069002803DA404246F00106A0613A
:10095000F00701D026F010066C2D0BD0682D09D0C1
:100960004C2D39D06A2D35D0742D35D07A2D33D019
:1009700016E038E0E1682F4620468847B842054631
:1009800009D16C2F26D04FF48060E16806432046E1
:100990008847054604E06C2F1AD04FF48070064358
:1009A0000DB3A5F14100192802D8203546F40066A0
:1009B0004A462946204626604E46FFF75DFC80B138
:1009C00001280BD0F61D26F0070000F1080956E7B4
:1009D0004020E4E78020D8E70020D6E706F10409AC
:1009E0004DE7284652E7206ABDE8F09F64250000E5
:1009F00030B5B0F10A0271F100034FEA900E4EEAF1
:100A0000817EB0EB0E0061EB91014FEA101E4EEAC1
:100A1000017E10EB0E0041EB11114FEA102E4EEA51
:100A2000016E10EB0E0041EB11214FEA104E4EEA21
:100A3000014E10EB0E0041EB1141401841F1000155
:100A40004FEAD00040EA41704FEAD1014FEA8104F9
:100A500044EA907410EB800544EB01046D1944EBFB
:100A60000404521BA3414FF0000348BF0A3200D5D3
:100A700030BD401C41F1000130BD2DE9F0470D466D
:100A800099469246044600F124080168880604D578
:100A9000E06921F01001216000E00120A84201DDA1
:100AA000471B00E00027A1697A1902EB0900081A28
:100AB000A0612078C00602D42046FFF7F3FC002690
:100AC00008E0D4E901211AF806009047206A401C8A
:100AD000761C20624E45F4DB2078C0060AD52046FD
:100AE000FFF7E0FC06E0D4E9012130209047206ABE
:100AF000401C2062381EA7F10107F4DC07E0D4E9AE
:100B0000012118F805009047206A401C2062281E29
:100B1000A5F10105F3DC2046FFF7DAFC207800069A
:100B200002D50220BDE8F0870120FBE72DE9FF4F49
:100B30000C461E464FF0FF378BB0D2E90001DDF8BE
:100B400060800A908A46C1F30A5505B93D460021E6
:100B500008464FF00000BAF1000F00F4400005DA3B
:100B600000EB80004FF4400101EA50004FEA905939
:100B7000B9F1010F00DDB9460A9850EA4A000ED0DB
:100B800044F61050A5F2FF3545432F14B8F1000F7D
:100B90001ED07542291E1EDDC9F100021CE0B8F10D
:100BA000010F4FF0000001D0302103E0F24305E0D7
:100BB0002154401CB042FBDB30460022002121546E
:100BC0000B99C1F80880C1E900200FB0BDE8F08F93
:100BD000BD1B6D1CDEE74A4600DA694206A800F03C
:100BE0000FFC06AB93E8070003AB83E80700504611
:100BF0000A9901F0B7FC8DE80700A0F500501F38F6
:100C000000900398002D0ADD42F21F014A46084475
:100C1000002303A90390684601F020FF09E0A0F536
:100C200000504A461F38002303A90390684601F08C
:100C30002AFF8DE807000004000C03D04FF0FF30BE
:100C4000410800E01046B8F1000F03D000220092E6
:100C500015461EE0751E05D4FFF7CAFE30326255F8
:100C60006D1EF9D5B3460122084302D000227F1C35
:100C700004E02078302801D100227F1E002A099745
:100C800084D01DE0112D07DAFFF7B2FE3032625535
:100C90006D1C50EA0102F5D1084302D00098C8B19A
:100CA0000EE00021681E05E0235C625C6354225460
:100CB000401E491C8142F7DBAB46A81B401E099031
:100CC000002004F80B000B98099AC0F80880C0E9CE
:100CD000002B7AE711264FF0000857E72DE9F04F77
:100CE00088460446D21D22F0070191B0D1E90001E7
:100CF000CDE90A0101F0FEFF02460B98C00F01D0BA
:100D00002D2007E02068810701D52B2002E020215B
:100D100001EAC000032A099001D0072A05DB034637
:100D20004146204600F02CFB0BE12078800601D5DF
:100D3000E06900E00620B8F1650F814606D0B8F101
:100D4000660F18D0B8F1670F70D131E00020B9F10B
:100D5000110F009001DB112301E009F101030AAA40
:100D600001A90CA8FFF7E2FEDDE90C70002609F1ED
:100D70000105834647E001204B4600904FF00047B5
:100D80000AAA01A90CA8FFF7D1FEDDE90DB00C9964
:100D90005D46002610B909F101000D18B9EB0500F8
:100DA00003D4C0F1FF3609F10105A5EB09002BE0E2
:100DB000B9F1010F01DA4FF001090020B9F1110F6B
:100DC0000090484601DD112300E003460AAA01A96C
:100DD0000CA8FFF7ABFEDDE90C704D4600268346FC
:100DE000207800070AD4AB4500DA5D4601A8012D42
:100DF00004DD411911F8011C302907D04F4502DAF2
:100E000017F1040F04DA012082460FE06D1EEEE7B1
:100E1000002F02DCED1B3E4403E0781CA84200DDFD
:100E20007D1CB81B00F1010A4FF000472078000735
:100E300003D4AA4501DB4FF0FF3A0021B7F1004F80
:100E40000DF143088DF8431024D002202B23002FEE
:100E500001DA7F422D230A21021EA0F1010000DCED
:100E60005FB197FBF1FC97FBF1F201FB1C7C17468D
:100E70000CF1300C08F801CDEEE7A8F10100037089
:100E80002188090501D5452100E06521A0F101086F
:100E900000F8011C09980FA9A1EB0807FF1D00B17C
:100EA0000120411901EBEA70A1693844081A401E7B
:100EB000A0612078C00602D42046FFF7F3FA099813
:100EC00028B1D4E901219047206A401C2062207893
:100ED000C00622D52046FFF7E5FA1EE0002E04DB0F
:100EE000B34502DD01A8805D00E03020D4E9012196
:100EF0009047206A401C2062761CAAF101005FEA3C
:100F0000000A0AD100F038FAC0680168405CD4E9F0
:100F100001219047206A401C2062281EA5F101058E
:100F2000DCDC07E0D4E9012118F8010B9047206AC6
:100F3000401C2062381EA7F10107F3DC2046FFF7B2
:100F4000C7FA032011B041E62DE9F04F04460D46E3
:100F5000D21D22F0070089B0D0E9009748463946F3
:100F600001F0C8FE0246F80F01D02D2307E02068EB
:100F7000810701D52B2302E0202101EAC0038DF86F
:100F800020300BB1012000E00020032A824601D06E
:100F9000072A04DB2946204600F0F2F93FE12078D9
:100FA000800601D40D2500E0E569C7F30A560D2D32
:100FB00049DA00214FEA175B08464FF00000002F86
:100FC00000F4400007DA00EB80004FF4400100EB32
:100FD000D07001EA60008115012901DD4FF0FF3179
:100FE00000224FEA850CBCF1180F06D31346ACF172
:100FF00018004FF08052C24003E04FF4801323FAF0
:101000000CF30CF10C0CBCF1200F04D3ACF1200C50
:1010100009FA0CF001E007FA0CF000294FF0004843
:1010200001DD18B90FE00ED140450CD319EB0209D0
:101030005F4121B9404502D19F4329EA0209BBEB38
:10104000175F00D0761C2088000502D57B487844C5
:1010500002E07A487844193808AA302302F80A30A6
:10106000037C0AF10101002E0AF1020A53546A4678
:1010700002DC4FF0300101E04FF031014FF0010888
:101080008DF8001002D0A6F2FF3603E059EA4701BE
:1010900000D06B4E002D02DC2178090704D54FF0FB
:1010A00002082E218DF80110C44600210BE0C7F381
:1010B00003433F01C35C491C6D1E02F8083005293B
:1010C00008F1010801DA002DF1DC00210CE000EB51
:1010D0001973491C1B786D1E082902F808304FEA65
:1010E000091908F1010801DA002DF0DC21688B06EE
:1010F00002D516E0A8F10108E04505DD02EB080382
:1011000013F8013C302BF5D0B8F1000F09DD02EBEC
:10111000080313F8013C2E2B03D1090701D4A8F1D1
:101120000108002D05DD3E2102F808106D1E08F1B2
:101130000108407C002E02F8080008F1010804DADA
:101140002D20764202F8080002E02B2002F8080069
:101150000A214FF47A70864208F101080BDB96FBF6
:10116000F0F3303302F8083096FBF0F308F1010891
:1011700000FB136601E0642E0CDB642096FBF0F3A9
:10118000303302F8083096FBF0F308F1010800FB59
:10119000136601E00A2E06DB96FBF1F0303002F810
:1011A000080008F1010896FBF1F001FB10603030F7
:1011B00002F80800A16908F1010808EB050202EB3A
:1011C0000A00081AA0612078C00602D42046FFF762
:1011D00069F9216A08AE01EB0A00206204E0D4E953
:1011E000012116F8010B9047BAF1010AF7D22078D5
:1011F000C00602D52046FFF755F96E4609E016F8FD
:10120000010B3E280FD0D4E901219047206A401CF1
:101210002062B8F10108F2D22046FFF759F909B06F
:101220000320BDE8F08F206A2844206203E0D4E95F
:101230000121302090476D1EEBD3F8E7B21D00006E
:1012400002FCFFFF01694A1C02610878704700B583
:101250008FB0CDE901310021059105497944CDE9EF
:10126000031011466846FFF7FFFA0FB000BD0000FB
:10127000E5FFFFFF10B5436913B1AFF3008001E054
:10128000FFF749F9012010BD127800F124010A701E
:1012900000224A700122EDE711684FF0FF32E9E7C2
:1012A00010B5436913B1AFF3008001E0FFF7BEF959
:1012B000012010BD128800F1240182840022C28422
:1012C0000122EDE711684FF0FF32E9E7007B00F003
:1012D000800070472DE9F04116460C46054600F0A7
:1012E00043F8036893F80101012807D0FF2C12D8B6
:1012F000185D80B101202C70BDE8F081D3F80701A2
:101300003246214603F20713C7182846BC46BDE8FB
:10131000F041002360474FF0FF30EDE7754600F0E5
:10132000EBF8AE4605006946534620F007008546B7
:1013300018B020B5FFF71AF8BDE820404FF00006BE
:101340004FF000074FF000084FF0000BAC46ACE840
:10135000C009ACE8C009ACE8C009ACE8C00921F09C
:1013600007018D467047000010B500F005F8001D1C
:1013700010BD00BFED19000000487047300000208C
:101380002DE9F0411F46044603260168072A01F4AF
:10139000006004DB08B116A505E016A503E008B15E
:1013A00015A500E015A521F010002060A069C01E61
:1013B000A0610FB1401EA0612046FFF773F84FB146
:1013C000D4E9012138469047206A401C2062C01CA5
:1013D000206206E0206AFAE7D4E9012115F8010B42
:1013E0009047761EF8D22046FFF772F8BDE8F081EC
:1013F0004E414E006E616E00494E4600696E6600B9
:101400002DE9F047814616468AB0354878440DC824
:101410008DE80D0032487844801C03AC0DC884E888
:101420000D0041F69B300844372190FBF1F290FB10
:10143000F1F5A5F1800501FB12041B3C02D56442C5
:10144000012000E00020DFF898A080460027FA4441
:10145000AAF1BE0A0EE0E0070AD03246684607EB62
:10146000470101230AEB810101F00DFB8DE8070024
:1014700064107F1C002CEED1194F7F44AE3F19E061
:10148000E80715D007EB04100DF1180A90E80E00DC
:101490008AE80E00C068F04201D1981908903246DF
:1014A000012306A903A801F0EEFA03AB83E80700C5
:1014B0006D10641C002DE3D14FF0010332466946E4
:1014C000B8F1000F03A802D001F0C8FA01E001F062
:1014D000DAFAC9E90001C9F808200AB0BDE8F087C6
:1014E000841A000010B50446AFF300802046BDE822
:1014F0001040FEF726BF0000004870471000002093
:1015000030B44FF0013C50F8042B51F8043BCCFAB6
:1015100052F4D51A20D1FCB950F8042B51F8043BF1
:10152000CCFA52F4D51A17D1B4B950F8042B51F8AB
:10153000043BCCFA52F4D51A0ED16CB950F8042BF6
:1015400051F8043BCCFA52F4D51A05D1002CDAD06C
:1015500030BC4FF00000704729BAB1FA81F111F0A8
:101560001801D1F120008440F2D1CA40CB4012F0E2
:10157000FF0213F0FF0330BCD01A704780B582B071
:10158000019000F02BF80090FFE700F027F8009999
:10159000401A0199884202D2FFE700BFF5E702B086
:1015A00080BD000072B6FFE700BFFDE780B500F028
:1015B00087FA40F20000C2F20000006844F6D351FE
:1015C000C1F26201A0FB0110800900F047FA18B1D6
:1015D000FFE7FFF7E7FFFFE780BD000040F2CC0028
:1015E000C2F200000068704780B541F20000C4F20A
:1015F0000200016841F4807101604FF4806100F0E5
:1016000061FF002000F0ACF941F20800C4F20200D2
:10161000012101600C21042200F07CFF00F0DAFAC5
:1016200080BD000080B58AB005A800F031F940F215
:10163000D000C2F200000078022801D0FFE7A6E047
:10164000079841F29311884204D8FFE7012000F087
:10165000F5FD9CE0099840F6D961884204D3FFE784
:10166000022000F0EBFD92E00898B0F5E17F04D98C
:10167000FFE7032000F0E2FD89E040F20800C2F23B
:101680000000006840F6E4410191A0FB0101079AC7
:101690000023FEF77EFE0146019803910999401A46
:1016A0000490049800EB400048F21F51C5F2EB1182
:1016B00050FB01F1481100EBD17240F2C800C2F2B8
:1016C0000000016811440160006840F6B9318842A9
:1016D00008DBFFE740F2C801C2F2000140F6B83073
:1016E000086016E040F2C800C2F2000000684FF245
:1016F0004741CFF6FF7188420ADCFFE740F2C8019C
:10170000C2F200014FF24840CFF6FF700860FFE7D9
:10171000FFE7039804995A22514348F21F52C5F239
:10172000EB1251FB02F2511101EBD271084440F26D
:10173000C801C2F200010968084402900898B0F597
:10174000967F0AD9FFE70898A0F59670C0EB0011C4
:101750000298A0EB81000290FFE70298B0F1FF3FF2
:1017600003DCFFE7002002900DE00298009000F0FB
:1017700005FD01460098884204DDFFE700F0FEFC0D
:101780000290FFE7FFE7029800F026FCFFE70AB0AF
:1017900080BD000083B08DF807009DF8070001466A
:1017A0000091042823D80099DFE801F003090F1500
:1017B0001B0043F21000C0F6000002901DE042F64C
:1017C000EE70C0F60000029017E042F6FF70C0F61F
:1017D0000000029011E043F22B00C0F600000290DE
:1017E0000BE043F23D00C0F60000029005E043F23A
:1017F0001D00C0F600000290FFE7029803B070479A
:1018000040F20400C2F200000068704740F2C400D9
:10181000C2F200000078704740F20800C2F20000F7
:101820000068704740F2D000C2F2000000787047B4
:1018300080B500F00DFB002000F006FE00F0FCFD7E
:1018400000F068FA00F0EEFB014640F2C500C2F27B
:10185000000001700078C00720B1FFE7002000F011
:10186000A3FBFFE740F2D001C2F2000101200870A3
:1018700040F2C401C2F200010020087080BD0000E7
:1018800040F2C500C2F20000007800F0010070478D
:1018900080B586B00590022000F090FA0599088086
:1018A000032000F08BFA05994880042000F086FAA6
:1018B000059988800598008800F0A6FA049005989C
:1018C000408800F0A1FA03900598808800F09CFA07
:1018D0000290049840F68B01C0F20301019100F0E0
:1018E00099FD05998860039800F084FD0199059A97
:1018F000D060029800F08EFD0599086106B080BDA9
:1019000083B08DF807009DF8070001460091032879
:101910001CD80099DFE801F002080E1442F6E670C8
:10192000C0F60000029017E042F6E070C0F600003A
:10193000029011E043F21500C0F6000002900BE0A7
:1019400043F22500C0F60000029005E043F21D00BE
:10195000C0F600000290FFE7029803B07047000055
:1019600083B0029044F24020C0F20F00019042F296
:101970000001C4F20201086820F00F00029A10432F
:101980000860FFE742F20000C4F20200006800F0C5
:101990000F01029A00209142009006D0FFE70198C3
:1019A000002818BF01200090FFE70098C00720B171
:1019B000FFE7019801380190E4E70198002818BF7B
:1019C000012003B07047000080B582B0019000F0A4
:1019D000B1FA41F25800C4F20200016841F48021DA
:1019E0000160006844F60001C4F2000100200860B4
:1019F00044F60402C4F20002106044F60802C4F285
:101A00000002106040F20000C2F200000068019A7B
:101A100000EB5200B0FBF2F044F60C02C4F20002FC
:101A200010600D20086002B080BD000081B08DF80C
:101A30000300FFE744F61C00C4F200000068000643
:101A4000002802D4FFE700BFF4E79DF8030044F646
:101A50002801C4F20001086001B0704780B582B06F
:101A6000009000980138B0F1807F03D3FFE7012098
:101A7000019019E0009801384EF21401CEF20001F5
:101A800008604FF0FF300F2100F01CF94EF21801F2
:101A9000CEF20001002008604EF21002CEF20002E9
:101AA000072111600190FFE7019802B080BD00009E
:101AB00040F2CC01C2F200010868013008607047B2
:101AC00080B5FFF791FD41F25800C4F202000168B1
:101AD00041F080510160006847F20001C4F200014A
:101AE0000868012262F34A20086047F28001C4F2CC
:101AF0000001086820F48070086047F21400C4F206
:101B000000004FF4806100F0B7FC18B9FFE7FFF761
:101B10006BFD5DE00420FFF723FF18B9FFE7FFF737
:101B200063FD55E041F20000C4F20200016841F497
:101B3000807101604FF4806100F0C4FC18B9FFE7C8
:101B4000FFF752FD44E041F20000C4F202000168D8
:101B500021F0807101604FF0007100F08DFC18B928
:101B6000FFE7FFF741FD33E041F20C01C4F202014F
:101B700045F23250C0F20010086041F20000C4F299
:101B80000200016841F0807101604FF0007100F0C7
:101B900099FC18B9FFE7FFF727FD19E041F20800AB
:101BA000C4F20200032101600C22114600F0B2FCD5
:101BB00018B9FFE7FFF718FD0AE042F20001C4F28E
:101BC0000201086840F4E060086000F003F8FFE7F5
:101BD00080BD000088B042F20040C0F2F4000790DF
:101BE00041F20800C4F20200006800F00C00069008
:101BF00006980C2835D1FFE742F20040C0F2F4000D
:101C0000059041F20C00C4F20200006804909DF8B7
:101C10001010012000EB111003900498C0F306206F
:101C200002900498C0F3416001900199022000EBFA
:101C300041000090049800F00300032806D1FFE75C
:101C400041F20020C0F27A000590FFE70598039961
:101C5000B0FBF1F0029948430099B0FBF1F0079016
:101C60000AE00698082806D1FFE741F20020C0F2FA
:101C70007A000790FFE7FFE7079841F20801C4F2F6
:101C800002010968C9B20A0942F6AC61C0F6000156
:101C9000895CC84040F20001C2F20001086008B04F
:101CA000704700004EF68851CEF20001086840F4FB
:101CB000700008604EF60851CEF200014FF000604F
:101CC0000860704782B08DF8070000919DF9070009
:101CD00000280AD4FFE7009800019DF907104EF292
:101CE0000042CEF2000288540BE0009800019DF8FB
:101CF000071001F00F014EF61452CEF20002885484
:101D0000FFE702B07047000081B00090FFE700BF1E
:101D1000FDE7000080B582B041F24C00C4F2020041
:101D2000016841F400510160006840F20831C5F2D9
:101D30000001086840F4403008600821C5F2000145
:101D40000191086820F000500860086840F0805059
:101D500008600120FFF712FC0199086840F000407C
:101D60000860FFE70820C5F200000068C00F10B14E
:101D7000FFE700BFF6E70C21C5F200014FF48050E9
:101D800008601421C5F2000145F6403008604FF0AC
:101D9000A041012008600821C5F20001086840F058
:101DA00001000860FFE74FF0A0400068C00710B9CD
:101DB000FFE700BFF7E702B080BD000081B00090F0
:101DC000009880013021C5F2000108604FF0A04169
:101DD0000C2008600821C5F20001086840F00400EA
:101DE0000860FFE74FF0A04000684007002802D4D9
:101DF000FFE700BFF6E74020C5F2000000686FF380
:101E00001F3001B07047000081B0ADF80200BDF88E
:101E1000020040F6E44148431121C1F20101A0FB58
:101E20000110000A01B0704780B582B001900091A6
:101E300001980A2804D1FFE70D20FFF7F7FDFFE71F
:101E40009DF80400FFF7F2FD019802B080BD00008C
:101E500041F24C00C4F20200016841F00701016048
:101E600000684FF09041086840F0FC0008600C21C9
:101E7000C4F60001086820F0FC00086040F2004150
:101E8000C4F60001086820F070600860086840F03F
:101E90002060086040F20441C4F60001086820F4A4
:101EA0004050086040F20841C4F60001086840F064
:101EB0007060086040F20C41C4F60001086820F030
:101EC0007060086040F22441C4F60001086820F404
:101ED0007F000860086840F45D00086040F600017B
:101EE000C4F6000108684FF63F72C0F6FF7210405A
:101EF000086008684023C5F200031843086040F6F4
:101F00000401C4F6000108684CF208039843086015
:101F100040F60801C4F6000108688023CAF20003F5
:101F20001843086040F60C01C4F600010868104030
:101F30000860704741F24C00C4F20200016841F0B1
:101F400004010160006840F60001C4F60001086861
:101F500020F470000860086840F42000086040F633
:101F60000401C4F60001086820F44060086040F6EF
:101F70000801C4F60001086840F47000086040F6EB
:101F80000C01C4F60001086820F47000086040F6F7
:101F90002401C4F60001086820F47F400860086846
:101FA00040F4EE400860704781B08DF803009DF862
:101FB0000300C00738B1FFE746F69431C4F20101CF
:101FC0003020086006E046F69831C4F20101302066
:101FD0000860FFE701B0704780B582B001900198BA
:101FE000002803D2FFE7002001900DE00198009047
:101FF00000F0C4F801460098884204D9FFE700F0D9
:10200000BDF80190FFE7FFE7019846F69C11C4F286
:1020100001010860019840F20401C2F20001086069
:1020200002B080BD80B584B046F68010C4F20100D5
:10203000029041F26000C4F20200016841F0806148
:102040000160006846F69831C4F201013020086052
:1020500000F0B6F840F20801C2F20001086046F64E
:102060008C31C4F201014FF48030086046F6CC3167
:10207000C4F201010B20086000F05AF890B9FFE7A4
:1020800046F69831C4F201013020086046F600019E
:10209000C4F20101086820F40020086000208DF8D7
:1020A0000F0040E0029908200190086040F208000B
:1020B000C2F200000068029948610299002088611C
:1020C0000299C86100F05AF80199029A5062029A86
:1020D0004FF47A709062029A40F66E40C0F25E1041
:1020E0009063029A0420D063029A1164029A5164A8
:1020F00002998864029940F22010C0F220004866DC
:1021000046F6BC31C4F201014FF40010086046F6F7
:102110000001C4F20101086820F4002008600120D9
:102120008DF80F00FFE79DF80F0004B080BD0000A0
:1021300082B044F24020C0F20F000190FFE746F663
:102140008830C4F2010001680020C9030029009012
:1021500006D4FFE70198002818BF01200090FFE790
:102160000098C00720B1FFE7019801380190E6E729
:102170000198002818BF012002B0704781B045F6D1
:10218000C050009040F20800C2F2000000680B2826
:1021900012D3FFE7009840F20801C2F2000109687B
:1021A0000139884208D3FFE740F20800C2F200007C
:1021B000006801380090FFE7009801B07047000008
:1021C00080B584B040F20000C2F200000268D10E77
:1021D00048F2A060C0F2010010EB421041F1000192
:1021E00040F64052C0F2030200230093FEF7D1F8FC
:1021F0000246009801920A46019903920291029ABE
:102200000399D2F16302884105D3FFE700200390D0
:10221000642002900EE002990398B1F5803170F1CC
:10222000000006D3FFE7002003904FF6FF700290F6
:10223000FFE7FFE7029804B080BD000080B582B0E0
:102240008DF8070000200090FFF7AEFE0098FFF722
:10225000C3FE009846F60002C4F20102116821F4A0
:102260000021116000F0F0F89DF8070040F2C40171
:10227000C2F20001087040F2D001C2F20001032056
:10228000087002B080BD000070B596B000201590B7
:10229000149013901290FFE7129841F2FF11C0F2D0
:1022A0007A01884206D8FFE700BFFFE712980130A5
:1022B0001290F1E7FFF77AF94FF4E1300B90FFF756
:1022C00083FBFFF7B5FA42F64C70C0F60000FEF74C
:1022D000D9F80B9942F6F660C0F60000FEF7D2F886
:1022E00040F20000C2F20000016842F6B970C0F688
:1022F0000000FEF7C7F8FFF78FFA024642F6277094
:10230000C0F6000040F64051C0F20301FEF7BAF8F3
:10231000FFF7B6FA024642F6E070C0F6000042F659
:10232000D271C0F60001002A18BF014642F61870AB
:10233000C0F60000FEF7A6F842F6BC60C0F600004A
:10234000FEF7A0F8FFE7FFF749F9119011981499EB
:10235000401A28B1FFE711981490FFF763F9FFE7DF
:1023600011981399401AB0F5FA7F41D3FFE71198FD
:1023700013900CA8FFF78CFAFFF754FAFFF7C0FA96
:102380000690FFF743FAFFF705FA0790FFF778FA90
:10239000024642F6E071C0F6000142F6DC70C0F67B
:1023A0000000002A18BF084608900E980A900F985F
:1023B0000990109CFFF724FA0546FFF72DFA0699BD
:1023C000079A089BDDF824E006460A98EC46CCF80C
:1023D0001060CCF80C50CCF80840CCF804E0CCF8F5
:1023E000000042F67170C0F60000FEF74BF8FFE700
:1023F000A9E7000081B0009000984FF47A7148433B
:102400004BF69B51CBF2CA51A0FB0110400A01B020
:102410007047000080B582B001900091019844F2AD
:102420004021C0F20F01A0FB0101009A0023FDF73B
:10243000B0FF02B080BD000040F62801C4F60001E4
:102440004FF440400860704781B08DF803009DF85C
:102450000300C00738B1FFE740F61801C4F60001D9
:102460000820086006E040F62801C4F600010820B4
:102470000860FFE701B0704784B00390029144F216
:102480004020C0F20F000190FFE703980168029A14
:1024900000201142009006D0FFE70198002818BFE5
:1024A00001200090FFE70098C00720B1FFE70198E6
:1024B00001380190E9E70198002818BF012004B015
:1024C0007047000084B00390029144F24020C0F2B3
:1024D0000F000190FFE703980068029A00EA0201EA
:1024E00000209142009006D0FFE70198002818BF15
:1024F00001200090FFE70098C00720B1FFE7019896
:1025000001380190E7E70198002818BF012004B0C6
:102510007047000085B004900391029244F240207D
:10252000C0F20F000190FFE7049800680399014092
:10253000029A00209142009006D0FFE701980028FF
:1025400018BF01200090FFE70098C00720B1FFE707
:10255000019801380190E7E70198002818BF012091
:1025600005B070475FEA400C08BF91F0000F4FEADA
:102570008C234FEAC12243EA51514FEA1C5018BF45
:1025800000F5F0404FEA300018BF41F000415FEA2B
:102590006C5C00F02980BCF1FF3F08BF40F0804038
:1025A0007047130C06BF12044FF0100C4FF0000CD4
:1025B000130E04BF12020CF1080C130F04BF12011A
:1025C0000CF1040C930F04BF92000CF1020CD30F1A
:1025D00004BF52000CF1010C11464FF00002A0F1B3
:1025E0001F00A0EB0C00704711F0004F08BF7047B0
:1025F00031F000413FF4D5AF0B0C06BF09044FF09A
:10260000100C4FF0000C0B0E04BF09020CF1080C6B
:102610000B0F04BF09010CF1040C8B0F04BF8900E0
:102620000CF1020CCB0F04BF49000CF1010CCCF1F2
:10263000200322FA03F341EA030102FA0CF2A0EBB1
:102640000C0000F10100704723F07F4720F07F4C21
:1026500080EA030000F00040ACEB070303F57C5375
:1026600003F1FF032DE9804909B44FEA144324EA3A
:1026700003484FEA154B25EA0B4E0FF2042606EBF2
:1026800013273E7803FB0667C7F5000707FB06F62E
:102690004FEAD64606F102064FEA543707FB066CAE
:1026A000CCF1005C4FEA1C472CEA074C0CFB06F50A
:1026B00007FB06F404EB15464FEA961649085FEA55
:1026C000320234BF00204FF000404FEAD13706FB02
:1026D00007FC4FEA1C4C0CFB0BF7D21B03FB0CF75F
:1026E00061EB07010CFB0EF7B0EB074072EB1742F2
:1026F0000CFB08F734BFA2EB0742B2EB074261EBD9
:1027000017414FEA0C444FEA910706FB07FC4FEADA
:102710001C4C0CFB0BF7B0EBC74072EB573203FBC2
:102720000CF734BFA2EBC742B2EBC74261EB5731A3
:102730000CFB0EF7B0EBC70072EB57720CFB08F7FF
:1027400034BFA2EBC702B2EBC70261EB57714FEA8D
:10275000816141EA92114FEA826242EA90124FEAA5
:10276000806004EBCC04039F4FEAD13706FB07FCE3
:102770004FEA1C4C0CFB0BF7D21B03FB0CF761EB75
:1027800007010CFB0EF7B0EB074072EB17420CFB96
:1027900008F734BFA2EB0742B2EB074261EB1741E7
:1027A0004FEA8C5504EB9C244FEA910706FB07FC8B
:1027B0004FEA1C4C0CFB0BF7B0EBC74072EB5732E7
:1027C00003FB0CF734BFA2EBC742B2EBC74261EB8D
:1027D00057310CFB0EF7B0EBC70072EB57720CFBD6
:1027E00008F734BFA2EBC702B2EBC70261EB577127
:1027F0004FEA816141EA92114FEA826242EA901205
:102800004FEA806015EB4C2544F100044FEAD137C4
:1028100006FB07FC4FEA1C4C0CFB0BF7D21B03FB1F
:102820000CF761EB07010CFB0EF7B0EB074072EB06
:1028300017420CFB08F734BFA2EB0742B2EB07428A
:1028400061EB17414FEA813141EA92414FEA82320E
:1028500042EA90424FEA80304FEA0C7615EB1C15A5
:1028600044F1000448EA03434EEA0B484FF0000EDF
:10287000B2EB080C71EB030724BF624639464EEBFE
:102880000E0E4FF0000B0018524149414BEB0B0B61
:10289000B2EB080C71EB03077BF1000B24BF62461F
:1028A00039464EEB0E0E4FF0000B001852414941D5
:1028B0004BEB0B0BB2EB080C71EB03077BF1000B3E
:1028C00024BF624639464EEB0E0E51EA020718BF8E
:1028D00046F0010616EB0E7655F1000254F10001A8
:1028E00003D5BDE88901BDE80088BDE88901BDE8E0
:1028F0000048B619524141EB0101A3F101037047B1
:1029000080807F7E7D7C7B7A79787776767574732C
:10291000727171706F6E6E6D6C6C6B6A6A696868EB
:10292000676666656464636362616160605F5F5E81
:102930005E5D5D5C5C5B5B5A5A59595858575756F7
:10294000565555555454535352525251515050505C
:102950004F4F4F4E4E4D4D4D4C4C4C4B4B4B4A4AAE
:102960004A494949484848474747474646464545F2
:10297000454444444443434343424242424141412B
:102980009C46002B30D477002BD04FEA37071CB57C
:1029900003B44FF010004FF01001BAF1000F06D051
:1029A000BCF1000FDCBF40F0080040F008014FF020
:1029B00000000FBCBDE810400BF1010BBBF1010F93
:1029C00008BF5FEA170722BF12F1010211F10101EE
:1029D0004FF0004143F1000300F0004043EA0000E3
:1029E0007047F9D35708D0E746EA06464FEA16463D
:1029F00013F1400F1FDD13F1200FDFBF16430A460E
:102A0000002120335B42BED0C3F1200746EA0646D0
:102A10004FEA164602FA07F746EA070622FA03F2D9
:102A2000C3F1200701FA07F742EA070221FA03F18E
:102A30004FF00003A7E746EA020646EA06464FEAD9
:102A4000164646EA0106BCBF46EA0646360C4FF07B
:102A500000034FF000024FF0000194E72DE9804C95
:102A600070B49A46934691E8380007C831EA400CA2
:102A700048BF34EA430C03D5FFF7E6FDFFF780FFBC
:102A8000F0BCBDE8008C2DE9804C70B49A469346AA
:102A900091E8380007C810F0804F08BF13F0804F4E
:102AA00003D100F005F8FFF76BFFF0BCBDE8008C28
:102AB00020F07F4723F07F4C80EA030000F00040C5
:102AC00007EB0C03A3F57C53A3F1FE0392F0000F78
:102AD00000F0B38095F0000F00F077802DE90149F8
:102AE0004FEA114021EA00484FEA144624EA06471B
:102AF00000FB06FC08FB06F607FB08F818EB064887
:102B00004CEB164C00FB07F718EB07484CEB174053
:102B10004FEA124B22EA0B4E4FEA154625EA0647CA
:102B20000BFB06FC0EFB06F607FB0EFE1EEB064E2D
:102B30004CEB164C0BFB07F71EEB074E4CEB174B01
:102B400018EB0B0840F1000018EB0E0B58EB0008D7
:102B500040F100008F1A4FF000014FF000063CBF1B
:102B6000C943661B14BFB5EB040C00213CBFC9432D
:102B7000F61B4FEA174427EA04454FEA1C472CEAA4
:102B8000074C04FB076205FB07F70CFB05F616EB89
:102B9000074642EB174204FB0CFC16EB0C4642EBDB
:102BA0001C421BEB060658EB020241414EEA8E0E18
:102BB00046EA9E0601D5BDE80189B619524141EBAE
:102BC0000101A3F10103BDE801894FEA144524EA9C
:102BD00005464FEA114721EA074C05FB07F406FBBF
:102BE00007F70CFB06F111EB074144EB174405FB1B
:102BF0000CFC11EB0C4144EB1C444FEA124722EA57
:102C0000074C05FB07F206FB07F70CFB06F616EB75
:102C1000074642EB174205FB0CFC16EB0C4642EB59
:102C20001C456A1854F1000148BF7047B61952415B
:102C300041EB0101A3F10103704795F0000F37D07C
:102C40004FEA114221EA02464FEA144724EA074CB0
:102C500002FB07F106FB07F70CFB06F414EB074435
:102C600041EB174102FB0CFC14EB0C4441EB1C4103
:102C70004FEA154725EA074C02FB07F506FB07F765
:102C80000CFB06F616EB074645EB174502FB0CFC62
:102C900016EB0C4645EB1C42121951F1000148BFDE
:102CA0007047B619524141EB0101A3F1010370478E
:102CB0004FEA144524EA05464FEA114721EA074C3A
:102CC00005FB07F106FB07F70CFB06F212EB0742C8
:102CD00041EB174105FB0CFC12EB0C4251EB1C4184
:102CE0004FF0000648BF7047921841EB0101A3F175
:102CF0000103704703B401984100009850EAC120D5
:102D000018BF04204A0D18BF40F0010040F2FF72C6
:102D1000B2EB515F08BF40F00200012808BF052058
:102D200002B0704730380A2801D2012070470020D5
:102D30007047000010B500290AD00878002807D095
:102D400005487844FEF7DCFB002801D0002010BDC8
:102D50000248784410BD00002E0300002603000046
:102D600010B500290AD00878002807D00548784413
:102D7000FEF7C6FB002801D0002010BD02487844B1
:102D800010BD00001E03000016030000F1EE100A43
:102D90004FF6FF71C0F2C03120EA010040F04070F0
:102DA000E1EE100A7047FDF799BFFEF7CDB80000BD
:102DB0000000000000000000303132333435363777
:102DC000383941424344454640305800303132336F
:102DD000343536373839616263646566403078006F
:102DE00004000008000000000000000200010000D4
:102DF00010303132333435363738396162636465C7
:102E000066787000303132333435363738394142E4
:102E1000434445465850000002400000000000A016
:102E20000000000005400000000000C80000000095
:102E30000C4000000000409C000000001940000011
:102E40000020BCBE0000000034400000BFC91B8E43
:102E500000000004B5400000504BCFD06607E2CF21
:102E6000010000006C4100003E8251AADFEEA73451
:102E700001000000D9420000DCB5A0E23A301F9703
:102E8000FFFFFFFFB4450000FD25A0C8E9A3C14F27
:102E9000FFFFFFFFFF3F0000000000800000000078
:102EA000FF3F000000000080000000000000000064
:102EB000000000000102030406070809506F77654F
:102EC000722073746167653A2064697361626C652E
:102ED0006420696E206170705F636F6E6669672E33
:102EE000683B20414443206D6F6E69746F72206FA0
:102EF0006E6C792E0A00555341525433207265741A
:102F00006172676574207072696E74663A20256C10
:102F10007520626175640A00485254494D20444C42
:102F20004C3A2025730A0050574D3A20256C7520E5
:102F3000487A2C20706572696F643D256C75204855
:102F40005254494D207469636B730A000A422D473D
:102F5000343734452D44504F5731204443444320A7
:102F6000737461727465722070726F6A6563740A3B
:102F70000073746174653D2573206661756C743DE2
:102F8000257320687274696D3D25732076696E3DE6
:102F9000256C756D562069696E3D256C756D4120F7
:102FA000766F75743D256C756D5620647574793D2A
:102FB000256C752F256C750A0053797374656D4304
:102FC0006F7265436C6F636B3A20256C7520487A8D
:102FD0000A006E6F74207265616479006E6F742DE3
:102FE00072656164790073746F70706564007669EE
:102FF0006E20756E646572766F6C746167650076BD
:103000006F7574206F766572766F6C74616765009A
:103010006E6F6E650072756E6E696E6700756E6BB1
:103020006E6F776E006661756C7400696E70757492
:10303000206F76657263757272656E740068727463
:10304000696D20646C6C2074696D656F7574000027
:10305000A031000800000020100000003C02000821
:10306000B031000810000020C80600005C02000813
:103070001C00000043000000F8FFFFFF0C000000F0
:103080000E0000000F0000002E00000010010000E4
:1030900043000000F8FFFFFF004040404040404038
:1030A000404041414141414040404040404040401B
:1030B00040404040404040404005020202020202BF
:1030C000020202020202020202202020202020200E
:1030D0002020200202020202020290909090909022
:1030E00010101010101010101010101010101010E0
:1030F0001010101002020202020288888888888854
:10310000080808080808080808080808080808083F
:103110000808080802020202400000000000000047
:10312000000000000000000000000000000000009F
:10313000000000000000000000000000000000008F
:10314000000000000000000000000000000000007F
:10315000000000000000000000000000000000006F
:10316000000000000000000000000000000000005F
:10317000000000000000000000000000000000004F
:10318000000000000000000000000000000000003F
:10319000000000000000000000000000000000002F
:1031A0000024F40090010000406A000000000000CC
:04000005080001D915
:00000001FF
